:1000000019C033C032C031C030C02FC02EC02DC087
:100010002CC02BC02AC0CDC028C027C026C025C0F8
:1000200024C023C022C021C020C01FC01EC01DC0CC
:100030001CC01BC011241FBECFEFD2E0DEBFCDBF5E
:1000400011E0A0E0B1E0EAECF8E002C005900D920A
:10005000A630B107D9F711E0A6E0B1E001C01D92CA
:10006000AB35B107E1F77CD12EC4CACF8064809351
:100070007C0080917A00806480937A0080917A007D
:1000800086FDFCCF2091780030917900C901089558
:10009000CF93DF9380913A01803110F010923A01B2
:1000A00080913A01C82FD0E0CC0FDD1FCD5EDE4F2E
:1000B0002881398140E050E080910F01909110013A
:1000C000A0911101B0911201821B930BA40BB50BEF
:1000D00080930F0190931001A0931101B09312012E
:1000E00082E0C4DF9983888380913A01C82FD0E0F1
:1000F000CC0FDD1FFE01ED5EFE4F2081318140E01F
:1001000050E080910F0190911001A0911101B091E8
:100110001201820F931FA41FB51F80930F019093AC
:100120001001A0931101B0931201C55CDE4F28812C
:10013000398140E050E080910B0190910C01A09139
:100140000D01B0910E01821B930BA40BB50B809394
:100150000B0190930C01A0930D01B0930E0183E06D
:1001600085DF9983888320913A01E22FF0E0EE0F3A
:10017000FF1FE55CFE4F4081518160E070E080919F
:100180000B0190910C01A0910D01B0910E01840F13
:10019000951FA61FB71F80930B0190930C01A0938E
:1001A0000D01B0930E012F5F20933A01DF91CF91A3
:1001B00008951F920F920FB60F9211242F933F9321
:1001C0004F935F936F937F938F939F93AF93BF935F
:1001D000809106018823E1F0299A80918400909112
:1001E00085002091000130910101820F931F4496F8
:1001F00090938B0080938A0080E38093800080E45A
:100200008093820080E280938000109206012998FA
:100210008091070190910801A0910901B0910A0114
:100220000097A105B10581F480910201909103012D
:10023000A0910401B09105018093070190930801FA
:10024000A0930901B0930A018091070190910801E0
:10025000A0910901B0910A01803020E0920721E0CD
:10026000A20720E0B20718F49C01AD0113C08F3F34
:100270002FEF920721E0A20720E0B20728F02FEF2E
:100280003FEF40E050E006C09C01AD015695479518
:1002900037952795821B930BA40BB50B8093070111
:1002A00090930801A0930901B0930A01609188001E
:1002B00070918900620F731F7093890060938800AA
:1002C0000097A105B10509F581E0809306018091B1
:1002D00035018823D1F08091360190913701A091AA
:1002E0003801B09139018093020190930301A093EA
:1002F0000401B093050180913301909134019093F2
:1003000001018093000110923501BF91AF919F913F
:100310008F917F916F915F914F913F912F910F90AE
:100320000FBE0F901F901895E1E8F0E01082109238
:1003300085001092840080E38093800081E08083B8
:10034000109289001092880082E086BBEFE6F0E010
:1003500080818260808387E880937A007894089512
:10036000DF92EF92FF920F931F93CF93DF9380E87A
:10037000809361001092610086E084B9D5DFDD24AE
:10038000D394CCEDDFEF84DE809135018823D9F75B
:1003900060910F01709110018091110190911201F3
:1003A0007DD120E030E040E85DE32AD220E030EC6F
:1003B0004FE754E4DFD020E030E44CE955E420D2AC
:1003C0007B018C017F2D912F20E030E040E251E451
:1003D000CDD0882324F4EE24FF2400E211E460E869
:1003E00076E988E19BE42E2D3F2D402F512FC2D07E
:1003F00020E030E040E05FE355D024D16093360147
:1004000070933701809338019093390160910B010B
:1004100070910C0180910D0190910E013FD120E06F
:1004200030E040E85DE3ECD120E030EC4FE754E40D
:10043000A1D022E838EA4BEF57E3E2D17B018C01EF
:100440007F2D912F2DEB37E346E855E38FD088239E
:1004500034F4EDEBEE2E77E3F72E06E815E36E2D80
:100460007F2D802F912F20E836E948E15BE4C8D149
:1004700020E030E040E05FE315D0E4D07093340139
:100480006093330180913301909134012FEF8D3DC2
:10049000920720F0D0933401C0933301D0923501FC
:1004A00072CF5058BB27AA270ED070C161D130F04F
:1004B00066D120F031F49F3F11F41EF456C10EF4C2
:1004C000E095E7FB4CC1E92F72D180F3BA176207C0
:1004D00073078407950718F071F49EF58AC10EF42E
:1004E000E0950B2EBA2FA02D0B01B90190010C0144
:1004F000CA01A0011124FF27591B99F0593F50F45C
:10050000503E68F11A16F040A22F232F342F4427B3
:10051000585FF3CF469537952795A795F0405395AB
:10052000C9F77EF41F16BA0B620B730B840BBAF07B
:100530009150A1F0FF0FBB1F661F771F881FC2F7E6
:100540000EC0BA0F621F731F841F48F487957795FA
:100550006795B795F7959E3F08F0B3CF9395880FB1
:1005600008F09927EE0F979587950895D4D008F451
:1005700081E008950CD00AC102D140F0F9D030F0EA
:1005800021F45F3F19F0EBC0511134C1EEC00FD11F
:1005900098F39923C9F35523B1F3951B550BBB274A
:1005A000AA2762177307840738F09F5F5F4F220FF7
:1005B000331F441FAA1FA9F333D00E2E3AF0E0E8F0
:1005C00030D091505040E695001CCAF729D0FE2F3C
:1005D00027D0660F771F881FBB1F261737074807CE
:1005E000AB07B0E809F0BB0B802DBF01FF27935884
:1005F0005F4F2AF09E3F510568F0B1C0FBC05F3FDE
:10060000ECF3983EDCF3869577956795B795F7956B
:100610009F5FC9F7880F911D9695879597F9089563
:10062000E1E0660F771F881FBB1F621773078407FF
:10063000BA0720F0621B730B840BBA0BEE1F88F70E
:10064000E0950895BCD088F09F5790F0B92F992776
:10065000B751A0F0D1F0660F771F881F991F1AF0CD
:10066000BA95C9F712C0B13081F0C3D0B1E0089596
:10067000C0C0672F782F8827B85F39F0B93FCCF317
:10068000869577956795B395D9F73EF490958095C3
:10069000709561957F4F8F4F9F4F0895E89409C0E3
:1006A00097FB3EF490958095709561957F4F8F4FA5
:1006B0009F4F9923A9F0F92F96E9BB279395F695BB
:1006C000879577956795B795F111F8CFFAF4BB0F39
:1006D00011F460FF1BC06F5F7F4F8F4F9F4F16C09D
:1006E000882311F096E911C0772321F09EE8872F27
:1006F000762F05C0662371F096E8862F70E060E0E3
:100700002AF09A95660F771F881FDAF7880F96955B
:10071000879597F90895990F0008550FAA0BE0E8FF
:10072000FEEF16161706E807F907C0F012161306B3
:10073000E407F50798F0621B730B840B950B39F4F3
:100740000A2661F0232B242B252B21F408950A2659
:1007500009F4A140A6958FEF811D811D089597F999
:100760009F6780E870E060E008959FEF80EC089557
:1007700000240A9416161706180609060895002480
:100780000A9412161306140605060895092E0394FA
:10079000000C11F4882352F0BB0F40F4BF2B11F46E
:1007A00060FF04C06F5F7F4F8F4F9F4F089557FDCD
:1007B0009058440F551F59F05F3F71F04795880FCF
:1007C00097FB991F61F09F3F79F087950895121666
:1007D00013061406551FF2CF4695F1DF08C0161612
:1007E00017061806991FF1CF8695710561050894C3
:1007F0000895E894BB2766277727CB0197F90895DA
:100800000BD0C4CFB5DF28F0BADF18F0952309F07C
:10081000A6CFABCF1124EECFCADFA0F3959FD1F3C3
:10082000950F50E0551F629FF001729FBB27F00D9E
:10083000B11D639FAA27F00DB11DAA1F649F6627F3
:10084000B00DA11D661F829F2227B00DA11D621F42
:10085000739FB00DA11D621F839FA00D611D221FFC
:10086000749F3327A00D611D231F849F600D211DE0
:10087000822F762F6A2F11249F5750408AF0E1F083
:1008800088234AF0EE0FFF1FBB1F661F771F881FCC
:1008900091505040A9F79E3F510570F060CFAACF0C
:1008A0005F3FECF3983EDCF3869577956795B795B7
:1008B000F795E7959F5FC1F7FE2B880F911D9695E1
:0A08C000879597F90895F894FFCF8B
:0608CA00F401A08601000C
:00000001FF
